:100000000C94AC030C94E4030C94E4030C94E4030C
:100010000C94E4030C94E4030C94E4030C94E403C4
:100020000C94E4030C94E4030C94EC270C94BE2889
:100030000C94E4030C94E4030C94E4030C94E403A4
:100040000C94E4030C94E4030C94E4030C94E40394
:100050000C94E4030C9471230C94E4030C94E403D7
:100060000C94E4030C94E4030C94E4030C94E40374
:100070000C94E4030C94E4030C94E4030C94E40364
:100080000C94C3080C94E4030C94E4030C94E40370
:100090000C94E4030C94E4030C94E4030C94E40344
:1000A0000C94E4030C94E4030C94E4037B095D09D1
:1000B00060096309660969096C096F0972097509A4
:1000C0007809EB0AF10AF70AFC0A010B060B0B0B85
:1000D000100B150B1A0B1F0B240B290B2F0BCF1119
:1000E000CF11FB11FB1163128E138E138E1381122D
:1000F0001A132B132B132B2952294A2A52294A2A25
:100100009E29C1294A2A182A272A0F0E0D0C0B0AEC
:1001100009131415161718100605040302011B1CF9
:100120001D1E1F20333231302F2E2D3738393A3BE8
:100130003C2B2A2928272625FF4041424344FFFF24
:1001400049585968638269A26EC571E9FFFFFFFFD4
:1001500043FF49FF4FFF54FF59FF5DFF62FF74FFEC
:10016000FFFF00003DFF37FF31FF2CFF27FF23FF7C
:10017000FFFFFFFF375827681D8217A212C50FE93E
:10018000FFFFFFFFFFFFFFFFC0FFB7FFB1FFACFFA7
:10019000A7FFA3FF9EFFFFFFB758A7689D8297A206
:1001A00092C58FE98CFFFFFFFFFFFFFFC958D96899
:1001B000E382E9A2EEC5F1E9FFFFFFFFFFFFC9FF00
:1001C000CFFFD4FFD9FFDDFFFFFFFFFFFFFFFFFFE2
:1001D000681058104810381028101810FFFFFFFF43
:1001E000680058004800380028001800000000107F
:1001F000FFFFFFFF780088009800A800B800C80043
:10020000FFFFFFFF781088109810A810B810C810D2
:10021000FFFFFFFFFFFFFFFF7030583048303830DE
:10022000283018300030FFFF682058204820382040
:10023000282018200020FFFFFFFFFFFF78208820E4
:100240009820A820B820C820FFFFFFFFFFFF8830BC
:100250009830A830B830C830FFFFFFFFFFFF0034F0
:1002600044540024455500253556002636460027BF
:1002700037470028384800293949002A3A4A002BD4
:100280003B4B00A4948400A5958500A6968600A704
:10029000978700A8988800A9998900AA9A7900AB45
:1002A0008A7A009B8B7B003C4C5C002C4D5D002DC2
:1002B0003D5E002E3E4E002F3F4F0030405000313B
:1002C0004151003242520033435300AC9C8C00AD8C
:1002D0009D8D00AE9E8E00AF9F8F00B0A09000B1AC
:1002E000A19100B2A28100B3928200A39383013452
:1002F000445401244555012535560126364601272B
:1003000037470128384801293949012A3A4A012B3F
:100310003B4B01A4948401A5958501A6968601A76F
:10032000978701A8988801A9998901AA9A7901ABB0
:100330008A7A019B8B7B013C4C5C012C4D5D012D2D
:100340003D5E012E3E4E012F3F4F013040500131A6
:100350004151013242520133435301AC9C8C01ADF7
:100360009D8D01AE9E8E01AF9F8F01B0A09001B117
:10037000A19101B2A28101B3928201A393830100F2
:100380002B0014001A000800150017001C001800AC
:100390000C00120013002A000100290004001600BE
:1003A000070009000A000B000D000E000F003300CB
:1003B00034000100E1001D001B00060019000500CB
:1003C000110010003600370038002800010001003D
:1003D000E000E200E300105F2C000000115F50001D
:1003E000510052004F00010035021E021F02200280
:1003F00021022202230224022502260227022A00C9
:1004000001004C003A003B003C003D003E003F0034
:100410002D022E022F0230023102010001004000A5
:1004200041004200430044004500320264024A0099
:100430004D00010001000100010001000100010068
:10044000010000000100AB00AA00A900AE000100FD
:1004500035001E001F002000210022002300240080
:100460002500260027002A0001004C003A003B002E
:100470003C003D003E003F002D002E002F003000CC
:1004800031000100010040004100420043004400EF
:100490004500320064004B004E00010001000100E5
:1004A0000100010001000100010000000100AB009B
:1004B000AA00A900AE000100010001000100010036
:1004C0000100010001000100010001000100010024
:1004D0000100010001000100010001000100010014
:1004E0000100010001000100010001000100010004
:1004F00001000100010001000100010001000100F4
:1005000001000100010001000100010001000100E3
:1005100001000000010001000100010001000001D4
:1005200001010101010101010202020202020202B3
:100530000203030303030303030404040404040485
:100540000505050505060606060607070707070849
:10055000080808090909090A0A0A0B0B0B0C0C0CFC
:100560000D0D0D0E0E0E0F0F0F1010111111121296
:1005700013131414151516161717181819191A1A13
:100580001B1B1C1D1D1E1E1F202021222223242474
:10059000252626272829292A2B2C2D2D2E2F3031B0
:1005A0003232333435363738393A3B3C3D3E3F40C2
:1005B0004142434445464748494A4C4D4E4F5051AD
:1005C0005354555658595A5B5D5E5F616264656667
:1005D00068696B6C6D6F7072737577787A7B7D7EEE
:1005E0008082838587888A8C8E8F91939596989A3E
:1005F0009C9EA0A2A3A5A7A9ABADAFB1B3B5B7BA56
:10060000BCBEC0C2C4C6C9CBCDCFD1D4D6D8DBDD29
:10061000DFE2E4E7E9EBEEF0F3F5F8FAFDFF2203A1
:10062000520041004D004100200057004F00520091
:100630004B00530020004D00350030002D004100DC
:1006400000001603520041004D00410020005700F9
:100650004F0052004B00530000000403090409023C
:100660003B00020100A0FA0904000001030101009F
:100670000921110100012240000705810308000142
:1006800009040100010300000009211101000122F9
:100690006D00070582032000011201000200000026
:1006A0000841520A0501000102000105010980A16B
:1006B00001850319012AB700150126B700950175B8
:1006C000108100C0050C0901A101850419012AA0AF
:1006D00002150126A002950175108100C0050109CF
:1006E00006A1018506050719E029E71500250195F2
:1006F00008750181020507190029EF1500250195EC
:10070000F07501810205081901290595057501910A
:1007100002950175039101C005010906A1010507B4
:1007200019E029E715002501950875018102950159
:10073000750881010507190029FF150026FF00959E
:1007400006750881000508190129059505750191AF
:1007500002950175039101C011241FBECFEFDAE0AD
:10076000DEBFCDBF04B603FE18C080916A0490912D
:100770006B04A0916C04B0916D048730904BA7403E
:10078000B04B59F410926A0410926B0410926C04EE
:1007900010926D04E0E0F8E3099511E0A0E0B1E00B
:1007A000EAEAF7E502C005900D92A83AB107D9F739
:1007B00024E0A8EAB1E001C01D92AA36B207E1F731
:1007C0000E949C1F0C94D32B0C9400000E94B60432
:1007D0000C944B1E0F931F93CF93DF93EC018B016F
:1007E0000E94CD0AC0318FE5D80729F0C131EFE56D
:1007F000DE0749F01EC0F8018281882311F081E0F4
:1008000007C081E013C0F8018281882371F082E083
:100810000E94F21443E062E081E00E94790F80E0E0
:10082000DF91CF911F910F91089582E00E941315DF
:10083000F1CFB801CE01DF91CF911F910F910C94B0
:10084000D70ECF93C82F0E94FD048C2FCF910C940C
:10085000F70F81E00C94FA0480E00C94FA0483E230
:1008600090E00E94502B823281F484E290E00E945A
:10087000502B823051F485E290E00E94502B91E0A1
:10088000873109F090E0892F01C080E081700895E0
:100890000E942F04882319F00E94950902C00E942B
:1008A0009D090E94A5090E94E1040C94F404CF93D1
:1008B000C82F811102C06FEF01C062E283E290E0B5
:1008C0000E946E2BC11102C06FEF01C062E084E292
:1008D00090E00E946E2BC11102C06FEF01C067E172
:1008E00085E290E0CF910C946E2B0E94480481E049
:1008F0000E9457040C944D1EDB01E82FF0E0EE0F30
:10090000FF1FE253FE4F94919C933196E491119610
:10091000EC931197863131F48091050180FF02C07C
:1009200098509C930895E82FF0E0EE0FFF1FE25CD3
:10093000FE4F8491DB018C933196E4911196EC93F8
:100940000895843020F08FEFDA018C9308956D3094
:10095000D0F7E62FF0E0BDE08B9FE00DF11D1124F4
:10096000E65FFE4FE491DA01EC93089560E084E7DE
:100970000E94AD0D61E086E70E94AD0D60E084E766
:100980000E94C50D61E086E70C94C50DCF93DF93FF
:100990001F92CDB7DEB7AE014F5F5F4F0E94A1043B
:1009A000E981F0E0E553FD4F10821092AC01109206
:1009B000AD011092AE011092AF010F90DF91CF9177
:1009C00008958091AB0181110EC081E08093AB014D
:1009D0008DE0809391009FB7F89423E020939900D5
:1009E000809398009FBF0895E1E7F0E080818260E6
:1009F000808308958093B50108958093B40108958C
:100A00008091B0019091B101A091B201B091B30178
:100A100080739927AA27BB2724E0B695A7959795B9
:100A200087952A95D1F782309105A105B10571F01E
:100A300083309105A105B10569F040E00197A1055A
:100A4000B10511F060E008C06FEF02C04FEF60E049
:100A500080E003C04FEF6FEF8FEF0C94970C40E0F6
:100A600060E080E00C94970CE5E0F1E06581768130
:100A700082810E94CB0B482F872F0C94970C5F929A
:100A80006F927F928F929F92AF92BF92CF92DF929E
:100A9000EF92FF920F931F93CF93DF931F92CDB7E7
:100AA000DEB760910A0170910B01809107010E94ED
:100AB000CB0BE62E972E882E60910C0170910D01C4
:100AC000809107010E94CB0B762E672E582E85E071
:100AD000C82E81E0D82EF12CAA24A394B12C00E0DA
:100AE00010E0AE014F5F5F4F602F8F2D0E94A10479
:100AF00089818834C0F4F60125893689A501002E44
:100B000002C0440F551F0A94E2F72423352390E0D6
:100B1000232B21F4282D4E2D692D03C0252D472D83
:100B2000662D0E94500C0F5F1F4F0D301105C9F646
:100B3000F394F2E0CF0ED11C84E0F812D0CF0F90E6
:100B4000DF91CF911F910F91FF90EF90DF90CF90A9
:100B5000BF90AF909F908F907F906F905F9008951F
:100B6000DF92EF92FF920F931F93CF93DF9300D00A
:100B7000CDB7DEB780910C0190E020910A01821B75
:100B800091098038910514F09A9505C081382FEFAE
:100B900092070CF4939597FD0396959587959595F7
:100BA0008795182F80910D0190E020910B01821BF9
:100BB000910997FD03969595879595958795082FAB
:100BC000D0900701E12CF12CBE016F5F7F4F8E2D7D
:100BD0000E947C048A8182958F7060910A01819FB6
:100BE000600D112470910B01809F700D11248D2DCB
:100BF0000E94CB0B462F282F672FC7010E94500C55
:100C00008FEFE81AF80A28E4E216F104E9F60F90EB
:100C10000F90DF91CF911F910F91FF90EF90DF9098
:100C20000895AF92BF92CF92DF92EF92FF920F930F
:100C30001F93CF93DF93082F10910A0180910C012D
:100C400090E0811B910997FD039695958795959561
:100C50008795D82FB0900B0180910D0190E08B19F2
:100C6000910997FD03969595879595958795C82F3A
:100C70000E941A2B68E470E00E94922AE12CF12C69
:100C80006C01DD24011103C0EC14FD04C9F40E94C1
:100C90001A2B8370A12E8D9FA00C11240E941A2B59
:100CA00083707B2D8C9F700D11246A2D809107011C
:100CB0000E94CB0B462F282F672FC7010E94500C94
:100CC0008FEFE81AF80A88E4E816F104D9F6DF9104
:100CD000CF911F910F91FF90EF90DF90CF90BF9039
:100CE000AF900895CF92DF92EF92FF921F93CF9330
:100CF000DF938091B0019091B101A091B201B091C8
:100D0000B3010090090104C0880F991FAA1FBB1FDF
:100D10000A94D2F7182F8BECE82E82E0F82EC0E070
:100D2000D0E09FE3C92ED12CF70181917F01F4E03F
:100D30008F9FC0011124CA32D10551F0C334D105AF
:100D400039F02091050123FF09C0C434D10531F4E5
:100D50008091EF0224E0829FC0011124803491052C
:100D600020F4B601681B790B02C060E070E0610FEF
:100D70007FEF809107010E94CB0B462F282F672F12
:100D8000CE010E94500C2196C834D10569F6DF913E
:100D9000CF911F91FF90EF90DF90CF9008958F92A9
:100DA0009F92AF92BF92CF92DF92EF92FF920F93FA
:100DB0001F93CF93DF9300D0CDB7DEB78091B00102
:100DC0009091B101A091B201B091B30100900901DD
:100DD00004C0880F991FAA1FBB1F0A94D2F7B82E10
:100DE000A09007018BECE82E82E0F82E00E010E0E6
:100DF0009FE3C92ED12CF70181917F01F4E08F9FF1
:100E0000C00111240A32110551F00334110539F0E3
:100E10002091050123FF09C00434110531F48091AC
:100E2000EF0224E0829FC00111248034910520F458
:100E30004601881A990A02C0812C912CBE016F5F6D
:100E40007F4F802F0E947C0469816B0D680D7FEFBE
:100E50008A2D0E94CB0B462F282F672FC8010E9496
:100E6000500C0F5F1F4F0834110529F60F900F909B
:100E7000DF91CF911F910F91FF90EF90DF90CF9076
:100E8000BF90AF909F908F9008958F929F92AF9256
:100E9000BF92CF92DF92EF92FF920F931F93CF9367
:100EA000DF9300D0CDB7DEB78091B0019091B10152
:100EB000A091B201B091B3010090090104C0880F64
:100EC000991FAA1FBB1F0A94D2F7B82EA090070142
:100ED0008BECE82E82E0F82E00E010E09FE3C92EB4
:100EE000D12CF70181917F01F4E08F9FC001112483
:100EF0000A32110551F00334110539F02091050132
:100F000023FF09C00434110531F48091EF0224E07D
:100F1000829FC00111248034910520F44601881A73
:100F2000990A02C0812C912CBE016F5F7F4F802FE8
:100F30000E947C046A816B0D680D7FEF8A2D0E94F0
:100F4000CB0B462F282F672FC8010E94500C0F5F34
:100F50001F4F0834110529F60F900F90DF91CF91A4
:100F60001F910F91FF90EF90DF90CF90BF90AF90C7
:100F70009F908F900895EF92FF920F931F93CF93BE
:100F8000DF93F82E0E941A2B68E470E00E94922AE8
:100F9000C0E0D0E08C011127F11003C00C171D0731
:100FA00089F40E941A2BE82E0E941A2B6E2D782F9E
:100FB000809107010E94CB0B462F282F672FCE016F
:100FC0000E94500C2196C834D10531F7DF91CF91A2
:100FD0001F910F91FF90EF900895EF92FF920F9362
:100FE0001F93CF93DF9300D0CDB7DEB78091B001D0
:100FF0009091B101A091B201B091B30100900901AB
:1010000004C0880F991FAA1FBB1F0A94D2F7F82E9D
:10101000E090070100E010E0BE016F5F7F4F802F7E
:101020000E94930469816F0D7A818E2D0E94CB0BF3
:10103000462F282F672FC8010E94500C0F5F1F4FAB
:101040000834110549F70F900F90DF91CF911F9150
:101050000F91FF90EF900895EF92FF920F931F93DF
:10106000CF93DF9300D0CDB7DEB78091B0019091E0
:10107000B101A091B201B091B3010090090104C087
:10108000880F991FAA1FBB1F0A94D2F7F82EE09071
:10109000070100E010E0BE016F5F7F4F802F0E94CC
:1010A000930469816F0D67FD6095669566958091E3
:1010B0000A01680F7A81769571588E2D0E94CB0BAC
:1010C000462F282F672FC8010E94500C0F5F1F4F1B
:1010D0000834110501F70F900F90DF91CF911F9108
:1010E0000F91FF90EF900895CF93C82F8091070143
:1010F0000E94CB0BCE3F29F4482F872FCF910C9421
:10110000970C282F462F672F8C2F90E0CF910C94AF
:10111000500C809110018F3F51F09091B40191FFDC
:1011200006C060910E0170910F010E94740883E067
:101130000E94D214882349F0809119018F3F11F148
:1011400060911701709118011BC082E00E94D214B7
:10115000882349F0809116018F3FA1F0609114011E
:10116000709115010DC081E00E94D214882351F0C6
:10117000809113018F3F31F0609111017091120144
:101180000C94740808951F920F920FB60F921124B9
:101190000F931F932F933F934F935F936F937F937F
:1011A0008F939F93AF93BF93CF93EF93FF938091D0
:1011B000AA01843120F48F5F8093AA01A2C080919C
:1011C000B0019091B101A091B201B091B30101962B
:1011D000A11DB11D8093B0019093B101A093B20104
:1011E000B093B3018091AC019091AD01A091AE019B
:1011F000B091AF018F3F2FEF9207A207B20759F0CE
:101200000196A11DB11D8093AC019093AD01A093F7
:10121000AE01B093AF01EBECF2E080818F3F11F0B3
:101220008F5F8083319683E0E331F807B1F7E09177
:101230000801EF3F19F40E94000563C08091B501D9
:10124000882321F08091050185FD1EC08091060153
:101250008823E1F020EB34E0829FA001839F500DB2
:101260001124052E000C660B770B81E00091AC0178
:101270001091AD012091AE013091AF01401751079F
:101280006207730720F002C081E001C080E0C82F30
:10129000C17080FDE0E081E0909104019E1301C0E7
:1012A00080E0E09304014E2F50E04B30510518F5DB
:1012B000FA01EA5AFF4F0C94C82A0E9434051DC057
:1012C0000E943F051AC00E94B00517C00E94110677
:1012D00014C00E94720611C00E94CF060EC00E9468
:1012E00045070BC00E94BB0708C00E94ED0705C060
:1012F0000E942C0802C00E942F05C11102C00E944A
:101300008908FF91EF91CF91BF91AF919F918F91FC
:101310007F916F915F914F913F912F911F910F910D
:101320000F900FBE0F901F9018954FE150E067E2AD
:1013300070E085E091E00C94402B4FE150E067E2D3
:1013400070E085E091E00C945E2BCF93DF930E94D8
:10135000F70D84E70E94000C86E70E94000CC0E0B5
:10136000D0E060E06170262F462F8C2F0E94B10CD8
:101370002196C834D10509F1CE0101979E0127506D
:1013800031092230310568F3877F4097029748F38F
:10139000CE0181978430910520F3CC32D10509F339
:1013A000439783309105E8F2099783309105C8F29D
:1013B00061E008970397B0F6D4CF60E084E70E941D
:1013C000C50D61E086E70E94C50DEBECF2E083E11C
:1013D00093E02FEF21938E179F07E1F7DF91CF91D5
:1013E00008958091080190E001968B30910514F0EA
:1013F0008AE090E0809308010C949D098091080197
:1014000090E0019797FF02C080E090E08B3091055B
:1014100014F08AE090E0809308010C949D0980917B
:10142000090190E001968430910514F083E090E08A
:10143000809309010C949D098091090190E0019726
:1014400097FF02C080E090E08430910514F083E0C3
:1014500090E0809309010C949D098091070190E030
:1014600008968F3F910519F014F08FEF90E080936C
:1014700007010C949D098091070190E0089797FF60
:1014800002C080E090E08F3F910519F014F08FEFDB
:1014900090E0809307010C949D0980910A0190E0EF
:1014A00008968F3F910519F014F08FEF90E080932C
:1014B0000A010C949D0980910A0190E0089797FF1A
:1014C00002C080E090E08F3F910519F014F08FEF9B
:1014D00090E080930A010C949D0980910B0190E0AB
:1014E00008968F3F910519F014F08FEF90E08093EC
:1014F0000B010C949D0980910B0190E0089797FFD8
:1015000002C080E090E08F3F910519F014F08FEF5A
:1015100090E080930B010C949D0980910C0190E068
:1015200008968F3F910519F014F08FEF90E08093AB
:101530000C010C949D0980910C0190E0089797FF95
:1015400002C080E090E08F3F910519F014F08FEF1A
:1015500090E080930C010C949D0980910D0190E026
:1015600008968F3F910519F014F08FEF90E080936B
:101570000D010C949D0980910D0190E0089797FF53
:1015800002C080E090E08F3F910519F014F08FEFDA
:1015900090E080930D010C949D090F931F93CF93BE
:1015A000DF93EC018B01DB0112968C91129788235B
:1015B00029F06C9111968C910E94C604FE01FF5592
:1015C000EE30F10508F050C0EF59FF4FD8011296E8
:1015D000CC910C94C82ACC2309F447C00E942D0A50
:1015E0003CC0CC2309F441C00E943B0A36C0CC2346
:1015F000E1F10E94F10931C0CC23B9F10E94FE094A
:101600002CC0CC2391F10E940F0A27C0CC2369F192
:101610000E941C0A22C0CC2341F10E944D0A1DC029
:10162000CC2319F10E945B0A18C0CC23F1F00E9470
:101630006D0A13C0CC23C9F00E947B0A16C0CC23CC
:10164000A1F00E948D0A09C0CC2379F00E949B0A68
:1016500004C0CC2351F00E94AD0AC0E006C0CC23E8
:1016600021F00E94BB0A01C0C1E08C2FDF91CF9115
:101670001F910F910895EF92FF920F931F93CF93B5
:10168000DF938B01682F11110AC0442329F0E82F42
:10169000F0E0E25EFA4F6491762F862F75C0212F1D
:1016A00030E0E82FF0E0442321F0E25EFA4FE491CD
:1016B000F0E046E0049FC0011124CFEFD0E0BE016E
:1016C0000E947E2A4BEA4603C001479F900D1124D9
:1016D000800F911D800F911D982F990F890FAE01DA
:1016E000421B530B4E9FD0014F9FB00D5E9FB00D1C
:1016F00011249B2F189FA0011124452F55278E01DF
:10170000041B150B0E9FA0010F9F500D1E9F500D27
:1017100011247E01E81AF108E29E8001E39E100D7B
:10172000F29E100D1124212F3327C21BD30BCE9F05
:101730009001CF9F300DDE9F300D11246230710576
:10174000A9F048F46115710569F061307105C9F4BB
:101750008B2F752F0DC06430710581F058F0663005
:10176000710579F47E2F8B2F932F0DC0832F7B2F44
:101770009E2F09C08E2F7B2F952F05C08E2F732F84
:1017800002C07E2F852F692FDF91CF911F910F917E
:10179000FF90EF90089541E00E943B0B0895E3E332
:1017A000F4E06083418324E630E042E050E0BF0192
:1017B000880F0C94AE0E0F931F93CF93DF93082FD7
:1017C000000FEB0114E210933304E4E3F4E0DE01D4
:1017D0008D91819384E0E434F807D1F724E630E07A
:1017E00041E150E063E374E0802F0E94AE0E105F91
:1017F0006096143B41F7DF91CF911F910F910895AF
:10180000CF93DF93C82F4BE06DEF0E94CF0B40E0EA
:101810006AE08C2F0E94CF0B8FE39CE90197F1F7D0
:1018200000C0000040E060E08C2F0E94CF0B40E041
:1018300061E08C2F0E94CF0B40E066E08C2F0E946D
:10184000CF0B40E06DEF8C2F0E94CF0BD0E040E03B
:101850006D2F8C2F0E94CF0BDF5FD231C1F740E09C
:101860006D2F8C2F0E94CF0BDF5FD432C1F740E089
:101870006D2F8C2F0E94CF0BDF5FD43BC1F74BE065
:101880006DEF8C2F0E94CF0B41E06AE08C2F0E94FD
:10189000CF0B40E06DEF8C2FDF91CF910C94CF0BED
:1018A000FF920F931F93CF93DF9300D000D0CDB75B
:1018B000DEB78834910588F5122F042FF62EBC016F
:1018C000660F771F660F771F625A7D4F44E050E026
:1018D000CE0101960E942A2B898183704A81282F8C
:1018E00030E050E9859FC00111248D5E9C4FFC01C2
:1018F000E40FF11DB497F0824B81FC01E40FF11D60
:10190000B49700834C81840F911DFC01B497108320
:10191000F901E452FE4F81E080830F900F900F9009
:101920000F90DF91CF911F910F91FF900895FF923B
:101930000F931F93CF93DF93182F062FF42EC0E041
:10194000D0E02F2D402F612FCE010E94500C219608
:10195000C834D105B1F7DF91CF911F910F91FF905E
:1019600008955F926F927F928F929F92AF92BF92F3
:10197000CF92DF92EF92FF920F931F93CF93DF935B
:1019800000D000D0CDB7DEB7862E942E522E24E0A4
:10199000829FC0011124BC01625A7D4F44E050E097
:1019A000CE0101960E942A2B2A8130E0C90184973A
:1019B000FC0197FD379673E0F595E7957A95E1F789
:1019C0004B8150E08A0104521109980117FF02C0AF
:1019D000295F3F4F63E0359527956A95E1F74C8184
:1019E00050E05A0164E2A61AB1083501B7FE04C0FE
:1019F0003A017DE1671A710843E0759467944A954E
:101A0000E1F758E0C52ED12CB6010E94922A7C0144
:101A1000C801B6010E94922A8C01C501B6010E943C
:101A2000922AFF274981FF24542F5370882081F088
:101A300062E1569FE00DF11D1124E854FE4F61E074
:101A400070E001C0660FEA94EAF75081652B10C080
:101A500072E1579FE00DF11D1124E854FE4F61E043
:101A600070E001C0660FEA94EAF760955081652343
:101A7000608333271127542F5370992089F062E136
:101A8000569F200D311D1124F901E854FE4F21E02D
:101A900030E001C0220F0A95EAF73081232B11C0F4
:101AA00072E1579F200D311D1124F901E854FE4FBA
:101AB00021E030E001C0220F0A95EAF7209530813D
:101AC0002323208377249927942F93709301552003
:101AD000A1F052E1959F200D311D1124F901E85428
:101AE000FE4F21E030E0B90102C0660F771F8A95F2
:101AF000E2F7CB019081892B14C072E1979F200DF2
:101B0000311D1124F901E854FE4F21E030E0B90104
:101B100002C0660F771F8A95E2F7CB01809590810E
:101B2000892380834370E42FF0E0EA54FE4F81E084
:101B300080830F900F900F900F90DF91CF911F91A6
:101B40000F91FF90EF90DF90CF90BF90AF909F905C
:101B50008F907F906F905F900895CF93DF93262FA3
:101B600030E0E901C452DE4F9881992351F090E9A9
:101B7000929FB001939F700D11246D5E7C4F0E9467
:101B8000DB0B1882DF91CF910895DF92EF92FF92E5
:101B90000F931F93CF93DF93262F30E0A9014A5470
:101BA0005E4F7A01FA01908191110AC0F70110820B
:101BB000DF91CF911F910F91FF90EF90DF900895EB
:101BC000D82EF2E16F9FE001112400E010E0F8014F
:101BD000EC0FFD1FE854FE4F4081602F8D2D0E94B9
:101BE000CF0B0F5F1F4F0231110589F7DFCF109226
:101BF000B9008CE08093B80008959F92AF92BF9295
:101C0000CF92DF92EF92FF920F931F93CF93DF93C8
:101C1000B82EEB010E944A236C01C431D10558F063
:101C2000CF3F8FEFD80759F0CE0164E170E00E94FA
:101C30007E2A7B0107C0EE24E394F12C03C025E04B
:101C4000E22EF12C84E8A82E94EA992E1092BC0082
:101C50009092BC000E944A238C018091BC0087FDB9
:101C600008C00E944A23801B910B8E159F05A8F384
:101C70002AC08091B900887F883041F08091B900F6
:101C8000887F803119F00FEF1FEF1FC0B092BB00AB
:101C9000A092BC000E944A238C018091BC0087FD69
:101CA00008C00E944A23801B910B8E159F05A8F344
:101CB0000AC08091B900887F883111F0803419F70B
:101CC00000E010E00EC00EEF1FEFCF3F8FEFD80700
:101CD00009F4BCCFC6010E9462238C179D0708F44B
:101CE000B5CFC801DF91CF911F910F91FF90EF9079
:101CF000DF90CF90BF90AF909F9008950F931F9368
:101D0000CF93DF93EB018093BB0084E88093BC000A
:101D10000E944A238C018091BC0087FD0EC0CF3FFA
:101D20008FEFD807C1F30E944A23801B910B8C17B9
:101D30009D0788F38EEF9FEF0CC02091B900287F9C
:101D400081E090E0283211F480E090E09195819557
:101D50009109DF91CF911F910F910895CF92DF925A
:101D6000EF92FF920F931F93CF93DF936B018A0142
:101D70007901B9010E94FD0DE6010C0D1D1DC01772
:101D8000D10761F424E92093BC00DF91CF911F912A
:101D90000F91FF90EF90DF90CF90089597FDF2CFD5
:101DA000B70189910E947E0EEACF81E0089581E01B
:101DB000089508950C94D90E1F93CF93DF9300D00C
:101DC00000D01F92CDB7DEB749835A836B83309121
:101DD000DF0189819A81311114C0662359F02223D1
:101DE00049F00E94E715182F682F89819A810E9477
:101DF000901503C00E94BB15182F69817A81812F2D
:101E000004C00E94E71569817A810F900F900F90AE
:101E10000F900F90DF91CF911F910C940B1DFC013F
:101E2000262F408151816281738184810C94DC0E64
:101E300081E00895CF93DF93EC0160E00E940F0FE3
:101E4000BE01DF91CF910C94DA0E8F929F92AF92E8
:101E5000BF92CF92DF92EF92FF920F931F936B018D
:101E60007C0181E090E0A0E0B0E04C015D0104C0A5
:101E7000880C991CAA1CBB1C4A95D2F7AC01BD0169
:101E800004C0440F551F661F771F2A95D2F74829B3
:101E900059296A297B2904C0880F991FAA1FBB1FD3
:101EA0000A95D2F78A019B010C211D212E213F2189
:101EB000401751076207730739F4BC01CD016C2943
:101EC0007D298E299F290AC080959095A095B0956F
:101ED000BC01CD016C217D218E219F211F910F918D
:101EE000FF90EF90DF90CF90BF90AF909F908F903A
:101EF00008950F93382F262F6091030270910402EA
:101F00008091050290910602042F432F0E94250F15
:101F10000F910C94AC140C9475040C94E603089582
:101F20000E941A140E948F0F2FEF84E39CE021502F
:101F300080409040E1F700C000000C9497230F937D
:101F40001F93CF93DF938C0161E00E940F0FEC0190
:101F5000B8010E94EA038823F1F1B801CE010E9482
:101F600095218823C1F1B801CE010E94A91F8823C1
:101F700091F1B801CE010E94F120882361F1F801AE
:101F80008281882309F1CB358DE5D807C1F050F463
:101F9000C115FCE5DF0781F0CF3DDC45A9F40E94C7
:101FA0001E1B19C0CC35EDE5DE0761F0CD35DD45F2
:101FB00059F40E94611A08C00E94900F0CC00E9440
:101FC0006A1A02C00E946D1AC801DF91CF911F9159
:101FD0000F910C94D50E80E0DF91CF911F910F915E
:101FE00008950C9429040E9406100C942C04089562
:101FF00081E008950C94F80F0895CF93C82F0E94A4
:1020000021048C2F0E94FA0FCF9108950E94F12194
:102010000C94FD0F0E94F1219091DE01891721F0AF
:102020008093DE010C94FD0F0895CF93DF93CDB71D
:10203000DEB72B970FB6F894DEBF0FBECDBF4F8330
:10204000588769877A878B8761110E94AD199E0135
:102050002F5F3F4F86E0F90111928A95E9F785E0FD
:10206000FE013796D90101900D928A95E1F7898199
:102070009A814C815D81452B31F09F3F31F491E095
:102080008F3F19F403C091E001C090E090FF09C0B8
:1020900049815A816B817C818D819E810E94CE18FD
:1020A00005C0C9010E94180F8111F2CF2B960FB6FF
:1020B000F894DEBF0FBECDBFDF91CF910895FC0134
:1020C000808191810E9429160895CF93882309F475
:1020D0009CC0C82F8238C1F40E94F12181FD95C0B7
:1020E00069E380912601909127010E94D9220E94E4
:1020F000CF192FEF81EE94E0215080409040E1F71E
:1021000000C0000069E319C0833801F50E94F12185
:1021100080FD7BC063E580912601909127010E949C
:10212000D9220E94CF192FEF81EE94E021508040F8
:102130009040E1F700C0000063E580912601909196
:1021400027010E94E422CF910C94CF198438C1F466
:102150000E94F12182FD59C067E48091260190918F
:1021600027010E94D9220E94CF192FEF81EE94E01F
:10217000215080409040E1F700C0000067E4DDCFCF
:102180008CEF8C0F813AD0F46C2F809126019091C6
:1021900027010E945922882349F06C2F8091260143
:1021A000909127010E94E4220E94CF196C2F809108
:1021B0002601909127010E94D922C5CF80E28C0F81
:1021C000883048F4C77081E001C0880FCA95EAF7EB
:1021D0000E949019B8CFEBE5EC0FE33040F4F0E04B
:1021E000ED59FE4F808190E0CF910C941722C85A90
:1021F000C73158F4EC2FF0E0EE0FFF1FEB5CFE4F01
:1022000080819181CF910C942D22CF9108958823C4
:1022100009F45BC0682F823879F40E94F12181FFB4
:1022200054C069E380912601909127010E94D92230
:102230000E94CF1969E310C08338B1F40E94F121E4
:1022400080FF43C063E580912601909127010E94A1
:10225000D9220E94CF1963E5809126019091270130
:102260000E94E4220C94CF19843879F40E94F12161
:1022700082FF2BC067E480912601909127010E9484
:10228000D9220E94CF1967E4E7CF8CEF860F813AFD
:1022900018F380E2860F883048F4677081E001C04F
:1022A000880F6A95EAF70E949619DCCF8BE5860FB6
:1022B000833020F480E090E00C941722685A673154
:1022C00020F480E090E00C942D2208951F93CF938A
:1022D000DF93182FEB010E946510209741F08FE9E2
:1022E0009FE00197F1F700C000002197F6CF812F02
:1022F000DF91CF911F910C940711893319F060E0A1
:1023000070E002C060E570E00C946611882321F053
:102310000E9490190C94CF190895882321F00E94EF
:1023200096190C94CF190895CF92DF92EF92FF92F5
:102330000F931F93CF93DF937C01D62FC72FFC0100
:102340001281058102950F700E9486198823B9F0C9
:102350001123A9F08C2F807F803421F080E28D0F33
:10236000883068F08091480482FD09C082E00E94B4
:102370002F1A0E94861991E0D82ED92601C0D12C9F
:10238000CC2EC2948FE0C8228C2D90E08C30910529
:1023900008F0C4C1FC01E159FF4F0C94C82A8C2FEE
:1023A000807FCF70882311F0C295C07F112399F0F0
:1023B000CC2309F49FC180E28D0F883010F0D11139
:1023C00004C08C2F0E94901903C08C2F0E94A0196A
:1023D0000E94CF198FC18D2F0E940711CC2309F4C1
:1023E0009DC180E28D0F883038F1DD2329F18C2FDB
:1023F0000E94A61924C08C2F807FCF70803211F0EC
:10240000C295C07FDD2319F0D130A1F13DC080918C
:10241000480482FF17C0112349F0CC2329F08C2FE8
:102420000E9490190E94CF1980E065C180E00E944F
:102430000711CC2309F472C18C2F0E9496190E94B7
:10244000CF196CC1112371F0002341F0013031F438
:102450000E94B0198C2B0E94B81960C10E94B0195B
:102460008C2B1DC0002319F0013009F457C10E94C4
:10247000C51925C0112321F0063008F04FC10EC048
:10248000053008F04BC11BC0112361F0002331F06F
:10249000F701858180FF2EC18F7085838C2F0E946C
:1024A00086113CC1002359F0D93309F034C1FFEF44
:1024B00007EE13E0F15000401040E1F72AC18C2FE5
:1024C0000E948D112BC18C2F86958695837019F0F3
:1024D000813061F023C1112321F08D2F9C2F937047
:1024E00002C080E090E00E94172220C1112321F059
:1024F0008D2F9C2F937002C080E090E00E942D22CF
:1025000015C18C2F837009F047C011110BC12D2FFD
:10251000229526952770220F220F6D2F6F70862F20
:1025200090E0A0E0B0E0022E04C0880F991FAA1F1F
:10253000BB1F0A94D2F7D4FF10C04FE050E060E018
:1025400070E004C0440F551F661F771F2A95D2F70D
:10255000409550956095709503C040E050E0BA01F9
:10256000C695C695C3708A019B01082B192B2A2B8F
:102570003B2BC901B801C23049F058F4C13019F001
:102580000E948614CFC00E947414CCC00E9498147C
:10259000C9C00E947214C6C0112319F08C2F81701B
:1025A00001C08695882309F4BDC02D2F229526955C
:1025B0002770220F220F6D2F6F70862F90E0A0E002
:1025C000B0E0022E04C0880F991FAA1FBB1F0A94F7
:1025D000D2F7D4FF10C04FE050E060E070E004C0DC
:1025E000440F551F661F771F2A95D2F740955095C7
:1025F0006095709503C040E050E0BA01C695C6955D
:10260000C3708A019B01082B192B2A2B3B2BC90174
:10261000B801C23049F058F4C13019F00E946B156E
:1026200081C00E9459157EC00E947D157BC00E940A
:10263000AC1478C0CF70112339F08C2F0E94F214A3
:102640008D2F0E9486116EC08D2F0E948D118C2FB0
:102650000E94131567C0D23F21F128F4D03F41F00A
:10266000D13FC1F043C0D33F19F1D43F79F03EC010
:10267000112341F0053008F051C08C2F8F710E945A
:1026800038154CC0063008F049C0F7CF8091480497
:1026900082FF18C0112339F08C2F8F710E94F21421
:1026A0003DC01123C9F38C2F8F710E94131536C0C2
:1026B000112329F08C2F8F710E94DD142FC00E94EE
:1026C000B8142CC0112349F0CF718C2F0E94F21442
:1026D00063E08C2F0E94141A21C081E00E942F1AFF
:1026E0000230E0F082E00E942F1A18C0112331F06E
:1026F000002391F28D2F0E94651010C0002399F2E3
:10270000D93349F41FEF27EE33E011502040304019
:10271000E1F700C000008D2F0E94071188EF8C0D9B
:10272000843020F40E94F1210E94FD0FDD20C9F0C9
:102730000E94821980FD15C0F70112820E947C1947
:102740000E94F214C7010E94D2130E947C19DF91EB
:10275000CF911F910F91FF90EF90DF90CF900C944D
:102760001315DF91CF911F910F91FF90EF90DF90A4
:10277000CF9008950F931F93CF93DF93EC0168815F
:1027800079818A810E9434168C010E948F150E94E3
:102790006014B801CE010E949411DF91CF911F9176
:1027A0000F910895CF93DF93EC01988189812B815C
:1027B0003C81232B31F08F3F31F481E09F3F19F4AE
:1027C00003C081E001C080E080FD1DC0CE010E94F9
:1027D0009F0F811110C00E9486198823A1F08A8161
:1027E000882389F08091480482FD0DC082E0DF914A
:1027F000CF910C942F1ACE010E94BA13CE01DF9113
:10280000CF910C941A0FDF91CF91089580E090E062
:102810000E94172280E090E00E942D220E94AD19B4
:102820000C94CF1980912601909127010E94EF22EC
:102830000C9406140E949D190C94121492959F708A
:10284000963079F010F4925001C09A50923068F4AA
:10285000803F69F018F4883E40F409C0843F29F4B1
:1028600006C0883E20F0813F11F080E0089581E0AD
:102870000895FC01808191810E9429160E941E14F6
:102880000895CF93DF9300D000D01F92CDB7DEB76D
:102890000F900F900F900F900F90DF91CF910895B0
:1028A000CF93DF9300D000D000D0CDB7DEB726960F
:1028B0000FB6F894DEBF0FBECDBFDF91CF91089564
:1028C000089508950C9461140C9462140E94641489
:1028D00060930702709308028093090290930A02A2
:1028E0000C9406140C9466140F931F930091070226
:1028F000109108022091090230910A02602B712B7D
:10290000822B932B1F910F910C9466140F931F939E
:1029100000910702109108022091090230910A02E9
:1029200060237123822393231F910F910C946614CB
:102930000F931F9300910702109108022091090242
:1029400030910A0260277127822793271F910F91E8
:102950000C9466140C9461140E94AA1460930302F0
:102960007093040280930502909306020C9406145F
:1029700060E070E0CB010C94AC1461157105810529
:10298000910529F481E0442361F080E00895DC01A1
:10299000CB0104C0B695A795979587954A95D2F730
:1029A00081700895482F6091030270910402809114
:1029B0000502909106020C94BD140F931F9341E001
:1029C00050E060E070E08A019B0104C0000F111F1D
:1029D000221F331F8A95D2F7C901B8011F910F91A9
:1029E0000C94AC140F931F9341E050E060E070E052
:1029F00004C0440F551F661F771F8A95D2F7809138
:102A0000030290910402A0910502B09106028A018E
:102A10009B01082B192B2A2B3B2BC901B8011F91B5
:102A20000F910C94AC140F931F9341E050E060E0C1
:102A300070E004C0440F551F661F771F8A95D2F7B8
:102A40004095509560957095809103029091040295
:102A5000A0910502B09106028A019B010823192367
:102A60002A233B23C901B8011F910F910C94AC1488
:102A70000F931F9341E050E060E070E004C0440F0A
:102A8000551F661F771F8A95D2F780910302909198
:102A90000402A0910502B09106028A019B01082759
:102AA00019272A273B27C901B8011F910F910C94C0
:102AB000AC140F931F930091030210910402209114
:102AC000050230910602602B712B822B932B1F91F4
:102AD0000F910C94AC140F931F930091030210916B
:102AE00004022091050230910602602371238223A3
:102AF00093231F910F910C94AC140F931F9300918B
:102B00000302109104022091050230910602602711
:102B10007127822793271F910F910C94AC1408956D
:102B20002DE0929F800D1124E82FE695E695E6951D
:102B3000877051E001C0550F8A95EAF785E0E89F5C
:102B4000F0011124E052FE4F20E030E070E04081BF
:102B5000CB01022E02C0969587950A94E2F7817008
:102B6000819584278523842781932F5F3F4F2530CC
:102B7000310569F708952DE0929F800D1124682F8B
:102B8000669566956695982F977085E0689FB00169
:102B9000112440E050E080E0FB01E40FF51FE0521B
:102BA000FE4F208130E0092E02C0369527950A9409
:102BB000E2F721703327042E01C0220F0A94EAF7AE
:102BC000822B4F5F5F4F4530510531F70895BF921B
:102BD000CF92DF92EF92FF920F931F93CF93DF93E9
:102BE0008C01C0900302D0900402E0900502F090A6
:102BF00006028091070290910802A0910902B0910B
:102C00000A02C82AD92AEA2AFB2ACFE1D0E0D70152
:102C1000C6010C2E04C0B695A795979587950A9482
:102C2000D2F780FD04C0219790F7B12C07C0BC2ECD
:102C3000B8018C2F0E941E1D0197A9F38B2DDF91E7
:102C4000CF911F910F91FF90EF90DF90CF90BF90A9
:102C50000895CF93DF93EC010E94E715BE010E9417
:102C60001E1DDF91CF9108951F93CF93DF93EB014A
:102C70009091DF01992321F0CB010E94291613C006
:102C8000882349F0CB010E94E715182F682FCE0149
:102C90000E94901504C0CB010E94BB15182FBE01E5
:102CA000812F0E941E1DDF91CF911F9108951F93C8
:102CB000CF93DF93C0910B0216E080910C02C817EE
:102CC00099F0D0E01C9FF0011D9FF00D1124E35FEF
:102CD000FD4F4081518162817381848195810E9481
:102CE00050142196C770E9CFDF91CF911F910895BD
:102CF00040913D0250913E0260913F02709140022E
:102D000080914102909142020C945014EF92FF92F4
:102D10000F931F93CF93DF938091420282958F7020
:102D200009F065C080913F02882309F460C080915A
:102D30000B02F0900C0210913D0200913E02609156
:102D400040027091410291E01F3F09F090E0C09174
:102D50002401D0912501292F96E0E92E8F1509F441
:102D600046C06115710521F00F3F21F030E003C02E
:102D700031E001C0322F90E030FD36C0E89EF00116
:102D8000E99EF00D1124DF01A35FBD4F11963C9128
:102D90001197301329C03C91311326C012963C91F3
:102DA0001297311121C013964D915C911497461BD7
:102DB000570B4C175D07C0F4809142028F70806101
:102DC00080934202EE5EFD4F80818F708061808330
:102DD0008DE392E00E94D213DF91CF911F910F916A
:102DE000FF90EF900C94571601968770B7CFDF9144
:102DF000CF911F910F91FF90EF9008959F92AF9206
:102E0000BF92CF92DF92EF92FF920F931F93CF93D7
:102E1000DF93CDB7DEB761970FB6F894DEBF0FBE74
:102E2000CDBF8C0185E0F801DE011D9601900D9269
:102E30008A95E1F7D8011296EC9090913D02E091CD
:102E40003E0220914002309141022115310531F0BE
:102E5000EF3F31F481E09F3F19F403C081E001C0EE
:102E600080E0B82FB1709B2E80FD47C1D8014C91F6
:102E700011965C9111971396AD90BC9014978DE3C9
:102E8000C82E82E0D82EF0903F02B501621B730B72
:102E90002091240130912501FF2009F4D9C08091AF
:102EA00042026217730708F095C0282F207F09F0AF
:102EB00052C05E1313C0491311C0FE2CE1100EC0A6
:102EC0008F708061809342020E947816C6010E9432
:102ED000D21380914202F80185834DC1AB2831F0B5
:102EE0005F3F31F481E04F3F19F403C081E001C03E
:102EF00080E080FD03C081E08E2502C080E090E08C
:102F0000F82FF170FF2E80FF1CC080910B022091E2
:102F10000C0236E0821709F40BC190E0389FF001F3
:102F2000399FF00D1124E35FFD4F6181561306C0F8
:102F30006081461303C06281E61203C00196877068
:102F4000E9CFFE2CEE2009F416C180914202816087
:102F50008093420254C05E1306C0491304C0E110BE
:102F600002C0F80199C0C8010E943914882361F198
:102F7000EE2051F120914202822F82958F7090E0D5
:102F8000029774F080913D0290913E0298878F8362
:102F90001986BB86AA862C87CE0107960E94D2137B
:102FA00086E0F801ADE3B2E001900D928A95E1F779
:102FB0000E9486160E9478160AC05E1711F1C80199
:102FC0000E94391481112CC0C8010E94D213FF2421
:102FD000F394D1C0282F207F81F77A2DB98AA88A4F
:102FE0006E2D89890E9441148DE392E00E94D213D4
:102FF00086E0D6011D928A95E9F70E947816F12C99
:10300000BAC04913DCCFE110DACFF8018583C801DB
:103010000E94D21386E0D6011D928A95E9F7ABC0D3
:10302000EE2091F220914202822F82958F7090E0E3
:1030300002970CF4B5CF80913D0290913E029A83A5
:1030400089831B82BD82AC822E83CE010196A6CFDE
:103050006217730708F044C0FE2CEE2009F4B4CFC9
:103060005E1330C049132EC02091420220FD21C0C2
:10307000822F82958F70482F50E041155105C9F07D
:10308000F80125834F30510541F08F5F982F9295BD
:10309000907F822F8F70892B8583C8010E94D21365
:1030A00086E0F801ADE3B2E001900D928A95E1F778
:1030B0003CC086E0F801ADE3B2E001900D928A9544
:1030C000E1F759C0C8010E943914811169CF80917C
:1030D0004202816080934202C8010E94D2134BC019
:1030E0007A2DB98AA88A6E2D89890E94411486E0BA
:1030F000D6011D928A95E9F718C0EE2009F464CF35
:10310000C8010E943914F82E882309F45DCF86E0A7
:10311000F801ADE3B2E001900D928A95E1F78DE3FD
:1031200092E00E945F100E9486160E94781623C0CB
:103130004D875E878D859E850E942916292F2295B1
:103140002F70223028F49F7039F0811105C00BC018
:10315000243028F49F7049F4805E883020F0C80144
:103160000E94D2139F2CF92C06C0D80115969C9171
:10317000907F91F7F8CF8F2D61960FB6F894DEBF50
:103180000FBECDBFDF91CF911F910F91FF90EF90B8
:10319000DF90CF90BF90AF909F9008951F93CF93F3
:1031A000DF93CDB7DEB72C970FB6F894DEBF0FBE16
:1031B000CDBF4F83588769877A878B879C87CE01DD
:1031C00007960E94FE168823D1F09F8188852A8564
:1031D0003B85232B31F08F3F31F481E09F3F19F481
:1031E00003C081E001C080E080FD47C04F81588569
:1031F00069857A858B859C850E9450143EC086E047
:10320000FE013796DE01119601900D928A95E1F745
:10321000FF81E8856A857B856115710531F0EF3F97
:1032200031F481E0FF3F19F403C081E001C080E088
:1032300080FD23C020910C0230E0C9010196877007
:10324000992740910B0250E084179507F1F1F9831B
:10325000EA837D836C8396E0929FD001939FB00DAB
:103260001124A35FBD4FFE01319601900D929A95F6
:10327000E1F780930C020E94571616E080910B0232
:1032800090910C02891771F1189FC0011124835F7E
:103290009D4F0E94FE16882329F1E0910B021E9F8C
:1032A000F0011124E35FFD4F408151816281738100
:1032B000848195810E94501480910B0290E00196C8
:1032C0008770992780930B02D9CF0E941A1410920D
:1032D0000C0210920B02EDE3F2E086E0DF011D929A
:1032E0008A95E9F72C960FB6F894DEBF0FBECDBFD6
:1032F000DF91CF911F910895809163028595859507
:103300008595089580916302877008959091630276
:10331000977081E009F480E0089580918602089515
:1033200090918602892B80938602089580959091D2
:10333000860289238093860208951092860208955A
:1033400090918502892B80938502089580959091B4
:10335000850289238093850208951092850208953D
:1033600080916402089508950C94B3190C94B419D3
:103370009091480492FD08C090916402981721F042
:10338000809364020C94B619089580916402882396
:1033900029F01092640280E00C94B6190895CF933E
:1033A000DF93E0912601F0912701809186028083CE
:1033B000E0912601F0912701908180918502892B6F
:1033C000808380916402882381F0E0912601F0914E
:1033D00027019081892B808380912601909127017C
:1033E0000E94432281110E94C519C0912601D091EB
:1033F000270140E250E063E472E0CE010E94332BEB
:10340000892B69F080E2FE01A3E4B2E001900D9205
:103410008A95E1F7CE01DF91CF910C94FD21DF91E8
:10342000CF9108950C94B3199091480492FD10C067
:1034300098E0899F90011124262B209363020E941B
:10344000F214809163028595859585950C94121AE6
:103450000C94F2141092630280E00C94121A2091E2
:1034600063028095822380936302982F977099F46A
:1034700030E0482F082E000C550B2417350759F063
:103480009091480492FD07C08595859585950E9489
:1034900013150C942A1A08959091480492FB222740
:1034A00020F9281769F080FB92F9909348048091E5
:1034B0004704909148040E949A1A82E00C942F1AB3
:1034C00008958091480482FB882780F991E089273C
:1034D0000C944C1A81E00C944C1A80E00C944C1A19
:1034E0006FEF7FEF80E090E00C948C2B80E090E019
:1034F0000E94582B21E0893E9E4F09F020E0822F48
:10350000089582E090E00C94502B83E090E00C94BE
:10351000502BCF9384E090E00E94502BC82F82E282
:1035200090E00E94502B2C2F30E0A901582BCA01AB
:10353000CF910895CF93C92F682F84E090E00E9427
:103540006E2B6C2F82E290E0CF910C946E2BAB012E
:10355000BC018FE090E00C94802BAB01BC0183E1B7
:1035600090E00C94802B60E070E0CB010C94AD1ADD
:1035700060E070E0CB010E94A71A0C94B31A69EEC8
:103580007EEF80E090E00E948C2B60E082E090E093
:103590000E946E2B60E083E090E00E946E2B109200
:1035A0000702109208021092090210920A0260E0CB
:1035B00084E090E00E946E2B60E082E290E00E9446
:1035C0006E2B60E085E090E00E946E2B60E086E06C
:1035D00090E00E946E2B6FEF87E090E00E946E2BD0
:1035E00040E050E0BA0188E090E00E94802B60E06B
:1035F0008DE090E00E946E2B40E050E0BA0188E13F
:1036000090E00E94802B60E087E190E00E946E2BAA
:1036100040E050E0BA018CE190E00E94802B60E035
:1036200070E080E290E00E948C2B40E050E0BA0114
:1036300088E190E00E94802B0C94B81A0C94BF1A79
:10364000682F8EE090E00C946E2B0E9456236093BE
:1036500093027093940280939502909396026093E4
:103660008F0270939002809391029093920208953A
:1036700085B7806885BF85B7806885BF089581E07C
:1036800008950C943F1B08950C94431B0C94431B0A
:103690000C94461B0C94431B0C944A1B0C94431B28
:1036A0000E94381B8AEF9DE10E94E7210E944E1B79
:1036B0000C944C1B0E94441B0C94431B0E94141E30
:1036C0000C94FC0F0E9441230E94F51E0E945E1B79
:1036D0000C94481B5F926F927F928F929F92AF9251
:1036E000BF92CF92DF92EF92FF920F931F93CF93EF
:1036F000DF93CDB7DEB72A970FB6F894DEBF0FBEC3
:10370000CDBF0E940A1FC82E81110E94251B37E8D9
:10371000832E32E0932E00E010E0502E802F0E9486
:10372000381E5C01F401619071904F016826792682
:1037300061147104B1F40F5F1F4F0430110569F774
:103740008FEF89838A831B820E944A238160782FAE
:103750009D838C8349815A816B818D810E941510D4
:103760003AC08091970281FD0E94411ED12CEE2427
:10377000E394F12CC3018E219F21892B29F10E9412
:10378000411B8823A9F0DE825F82AE20BF2081E04A
:10379000AB2809F480E088870E944A238160782F53
:1037A0009A8789874E815F8168858A850E94151076
:1037B000000F111FF801E957FD4F80819181E82624
:1037C000F926F182E08207C0D394EE0CFF1CFDE0E5
:1037D000DF12D0CFB0CF81E0C11001C080E02A96C7
:1037E0000FB6F894DEBF0FBECDBFDF91CF911F9112
:1037F0000F91FF90EF90DF90CF90BF90AF909F9090
:103800008F907F906F905F9008950E946A1B0C9438
:103810000A10CF93DF930E94231DEC01811522E54E
:103820009207E8F5811531E5930708F0B6C0883EA8
:10383000910528F5803E910508F0E9C0883A910588
:1038400070F4853A910508F07AC08130910509F449
:1038500073C008F4D9C0049708F0D9C0D5C08F3B15
:10386000910508F0D1C0C85AD0E0CC0FDD1FCA596D
:10387000DE4F0990D881C02DCE019464C9C0811556
:1038800040E5940708F069C0811550E4950708F0F9
:1038900060C09A9581159F4108F4B9C0B5C08115E3
:1038A00036E5930728F5811545E5940708F092C0A1
:1038B000811554E5950708F087C0AC014370552782
:1038C000282F26952695C115D34508F06CC081E0B8
:1038D00090E002C0880F991F4A95E2F740E2249FCA
:1038E00090011124EC01C22BD32BCE019C6890C017
:1038F00081152AE5920780F4811539E5930708F0D0
:1039000072C0811548E5940708F47EC0D82FCC27F3
:10391000CE01806F906A7CC090568115904208F06D
:1039200073C08D2F8F710E94B71DDD27D0628F71FC
:10393000AE01582BCA016CC081E090E069C0C55A45
:10394000D0E0CC56DE4F8881C82FD0E0CE01906405
:103950005FC0DF70CE01906A5BC074E0969587957A
:103960007A95E1F7282F23703C2F337081E090E0A7
:1039700002C0880F991F3A95E2F79C68AC01522B60
:103980009A019C2F9F709695969550E2959FE00125
:103990001124C9018C2B9D2B3BC0D82FCC27CE01E5
:1039A000816F906A35C081E090E002C0880F991F56
:1039B0004A95E2F750E2259F90011124EC01C22BB9
:1039C000D32BCE019A6824C0D82FCC27CE01846F88
:1039D000906A1EC00E94B71D8F7190E0D82FCC272F
:1039E000CE01906215C08F700E94B71D94E0D695ED
:1039F000C7959A95E1F7CF70D0E0DC2FCC27D0693E
:103A00009E01282BC90104C080E090E001C0CE01D6
:103A1000DF91CF91089524E3829FC0011124FC011E
:103A20002DE0729FE00DF11D1124E60FF11DEE0F48
:103A3000FF1FE258FC4F8591949108950E940B1D41
:103A40000E94091C08958238910569F1B0F4813310
:103A5000910509F46DC048F48932910509F463C0F9
:103A60008A32910509F469C008958533910509F4F6
:103A700055C089339105B9F00895833E910569F1E8
:103A800038F4803E9105B1F0823E910509F1089528
:103A9000863E9105A9F1873E9105B9F1843E9105D5
:103AA00009F064C023C02091470420FD4FC021FDD0
:103AB0004DC008958091470480FD44C08091480422
:103AC00080FF44C08091470484FD42C083EE4DC016
:103AD0008091470482FF38C0F5CF8091470482FD72
:103AE00033C08091480480FD31C0ECCF8091480400
:103AF00081FF32C08091470484FD2AC087EE35C023
:103B00008091470483FF26C0F5CF8091470483FD51
:103B100021C08091480481FD1FC0ECCF80914704F3
:103B200085FD1CC01DC08091470485FD19C016C0CD
:103B30008091470486FD16C017C08091470486FD1A
:103B400013C010C089E311C082EE0FC080EE0DC01B
:103B500080E00BC086EE09C084EE07C089E205C094
:103B600085E303C08AE201C081E390E0089590916B
:103B7000470492FF0DC0282F2871283019F4877F41
:103B8000846006C0282F2471243011F48B7F886054
:103B900093FF0DC0282F2871283119F4877E846186
:103BA00006C0282F2471243111F48B7E8861209166
:103BB000480420FF0DC0382F3871383019F4877F42
:103BC000816006C0382F3171313011F48E7F8860EA
:103BD00021FF0DC0282F2871283119F4877E8161BB
:103BE00006C0282F2171213111F48E7E886194FD49
:103BF000877E089580E008950C94701A0E940A1F31
:103C00008FE39CE90197F1F700C000000E940A1FB2
:103C100080E00E94381E80FF04C00E94FC1D0C94AE
:103C2000972308950C94FE1D0E94761A811102C0FC
:103C30000E941E1B0E94811A809397020E94891A7B
:103C400090934804809347040E94121E0E94851A94
:103C5000682F70E080E090E00E947214609103028F
:103C60007091040280910502909106020C94AA14AE
:103C7000E82FF0E0EE0FFF1FEF5AFB4F808191819C
:103C80000895089580EA8A95F1F7089500C008958F
:103C90000C94421E08950C944A1E0C944A1EF894EB
:103CA000E82FE295EF70F0E031A1282F2F7081E02E
:103CB00090E001C0880F2A95EAF7982F90959323FA
:103CC00091A392A1892B82A3789408950F931F93B7
:103CD000CF93DF93C4EAD1E089918F3F11F00E9426
:103CE0004F1E81E0C83AD807B9F7C7E9D1E004EA26
:103CF00011E089918F3F11F00E944F1E0C171D0794
:103D0000C1F7DF91CF911F910F910895BF92CF928C
:103D1000DF92EF92FF920F931F93CF93DF938C016B
:103D2000C62FD0E0CE018C559E4F6C01FC019081D6
:103D30009F3F09F450C0B62EF894E92FE295EF703A
:103D4000F0E081A19F7021E030E001C0220F9A9540
:103D5000EAF7822B81A382A12095282322A37894BD
:103D60000E94461EE7E9F1E044EA51E021E030E03C
:103D7000E12CF12C61916F3F89F0A62FA295AF70D5
:103D8000B0E090968C9190E06F7002C09595879509
:103D90006A95E2F780FD02C0C90102C080E090E0B0
:103DA000E82AF92A220F331F4E175F0719F7F60189
:103DB00080818F3F11F00E944F1E61E0E114F104F9
:103DC00009F460E08B2D0E94481ECC0FDD1FC00F50
:103DD000D11FF982E882DF91CF911F910F91FF905F
:103DE000EF90DF90CF90BF9008950E94661E88E00C
:103DF000E1E5F4E0DF01982F1D929A95E9F7E9E4F7
:103E0000F4E0DF011D928A95E9F784E00E94551FD6
:103E10000C948B0FFF920F931F93CF93DF93CDB72B
:103E2000DEB728970FB6F894DEBF0FBECDBF8E0168
:103E30000F5F1F4F88E0F80111928A95E9F7F12C86
:103E40006F2DC8010E94861EF394F4E0FF12F8CF94
:103E500048E050E0B80189E494E00E94332BFF244D
:103E6000F394009709F4F12C892B41F088E0F801D4
:103E7000A9E4B4E001900D928A95E1F72F2D44E07A
:103E800061E574E089E494E00E94561F0E948D0F62
:103E90008F2D28960FB6F894DEBF0FBECDBFDF91F1
:103EA000CF911F910F91FF9008950895FF920F9366
:103EB0001F93CF93DF93F82E092F162FD72FC42FE0
:103EC000222349F081E080939A020E944A23909332
:103ED00099028093980280919A028823D9F0809168
:103EE0009802909199020E946223059798F0EF2D15
:103EF000F02FA12FBD2F80E090E04C2F50E08417D1
:103F0000950734F4219131912D933D930196F7CF8C
:103F100010929A02DF91CF911F910F91FF90089517
:103F20000E9444250E94621B0C9450250E94542537
:103F30000E94051C0C946E250E9435230E942B259F
:103F40000E94501B0E94901F0E94961F0E945A1BA5
:103F5000FBCFCF93DF93EC01FB018281882309F42F
:103F60003CC1C430FDE5DF0760F4CB3F9CE5D907D9
:103F700088F49E0122503C452431310508F02EC1C1
:103F800009C0C236EDE5DE0729F0C63AFDE5DF07D8
:103F900009F024C10E94891A909348048093470431
:103FA000C1318CE5D80709F4C6C008F042C0C93059
:103FB000ECE5DE0709F49BC000F5C5308CE5D807B9
:103FC00009F485C078F4C330ECE5DE0709F478C065
:103FD00008F07AC0C230DC4509F0F5C08091470492
:103FE0008160EFC0C7309CE5D90709F478C008F0BC
:103FF0007AC0809147048061E4C0CD30FCE5DF07E2
:1040000009F487C058F4CB309CE5D90709F479C08E
:1040100008F07BC08091470488606FC0CF30FCE51A
:10402000DF0709F480C008F082C080914704877FD1
:10403000C8C0CE3F9CE5D90709F471C000F5C53171
:10404000FCE5DF0709F485C068F4C3319CE5D907B6
:1040500009F475C008F095C00E941A1480914704B5
:104060008F77AFC0CC3FFCE5DF07A9F108F054C063
:10407000CB3FDC4509F0A7C08091480440C0C23066
:10408000EDE5DE0709F489C058F4C1158DE5D807C0
:1040900009F45AC008F069C08091480482602FC0BA
:1040A000C236EDE5DE0709F47CC0C63AFDE5DF0760
:1040B00009F481C0C330DD4509F085C080E06EC0E1
:1040C0008091470482607DC08091470416C0809132
:1040D0004704886076C08091480482604FC0809118
:1040E000470480626EC08091470480646AC00E9469
:1040F0001A1480914704806864C0846062C0816043
:104100003DC0809147048E7F5CC0809147048D7FC5
:1041100058C08091470416C08091480418C080910F
:1041200048048D7F2BC0809147048F7E4AC08091C8
:1041300047048F7D46C0809147048F7B42C08091A9
:104140004704877F8B7F3DC0809148048D7F8E7FA1
:1041500015C08091470482FB222720F991E0922725
:1041600090FB82F990FB83F92CC080914804982F32
:10417000909591708E7F892B90FB81F980934804F4
:1041800022C00E941A148091470487FB222720F93D
:1041900091E0922790FB87F914C081E00E94201BD8
:1041A00012C08091470484FB222720F991E09227D6
:1041B00090FB84F906C080914704982F909590FB5E
:1041C00080F98093470480914704909148040E94AD
:1041D0009A1A0E941A1480E001C081E0DF91CF9109
:1041E0000895CF93DF9386319C4541F5EB010E9402
:1041F0008D19982F8A8120912601309127018823DB
:1042000079F09A7A81E009F480E080939B02911121
:1042100002C069E201C065E3C9010E94D9220AC057
:1042200080919B02811102C069E201C065E3C9016E
:104230000E94E4220E94CF1980E001C081E0DF915A
:10424000CF9108950F931F93CF93DF93C42FD22F55
:10425000FC0182818823C9F040939E020E944A2378
:1042600090939D0280939C0280E28C0F883008F02E
:1042700057C0C77081E001C0880FCA95EAF7DF9187
:10428000CF911F910F910C94861180919E0248133B
:1042900030C080919C0290919D020E946223883CD4
:1042A000910538F510E21D0FCD17B9F080E28C0FA3
:1042B000883040F4C77081E001C0880FCA95EAF7E2
:1042C0000E948D11183028F581E09D2F977001C054
:1042D000880F9A95EAF70E948611802F0E947D111F
:1042E0001830F0F4D77081E001C0880FDA95EAF752
:1042F0000AC080E28C0F883098F4C77081E001C05A
:10430000880FCA95EAF7DF91CF911F910F910C9416
:104310008D11802FDF91CF911F910F910C947D1102
:10432000DF91CF911F910F9108950F939C01CB01C5
:10433000243F4CE5340731F188F4293DFCE53F0783
:10434000D9F02A3D4CE5340779F1283D3C45A9F5E3
:1043500006E221EE41EE68ED7CE52BC0263FFCE550
:104360003F07E1F0A8F0273F3C4539F507E225EE8D
:1043700046EE67EF7CE51DC007E225EE45EE69EDF0
:104380007CE517C006E221EE40EE64EF7CE511C04B
:1043900007E225EE44EE65EF7CE50BC006E221EE78
:1043A00042EE66EF7CE505C008E221E045EE6AEDED
:1043B0007CE50E94222180E008C0FC0182818823E4
:1043C00019F010929E0201C081E00F910895909320
:1043D000A9018093A80108959093A4028093A30259
:1043E0000895E091A302F091A402309721F001908A
:1043F000F081E02D099480E00895E091A302F0910E
:10440000A402309799F020913401222359F0209191
:10441000470427FF07C0DC012C9111962C931197BC
:1044200026E02C930280F381E02D099408952091D9
:10443000A1023091A2022817390771F09093A202CD
:104440008093A102E091A302F091A402309721F0A1
:104450000680F781E02D0994089520919F02309104
:10446000A0022817390771F09093A00280939F0251
:10447000E091A302F091A402309721F00084F1852D
:10448000E02D09940895FC0132968091340188232F
:1044900031F08091470487FF02C09EE101C096E0A1
:1044A00080E0915028F021912223D9F38F5FF9CF3A
:1044B0000895662351F1209134012223E9F02091DF
:1044C000470427FF19C0462F4695469546954E311D
:1044D000E0F4677021E030E002C0220F331F6A95DC
:1044E000E2F7FC01E40FF11D828190E028233923DB
:1044F00081E0232B69F409C0FC01329608962191D2
:10450000621729F0E817F907D1F780E0089581E0F4
:1045100008959C01FC0132969FEF80E0419146177F
:1045200089F09F3F19F4411101C0982F8F5F8630A9
:10453000A9F79F3F39F0F901E90FF11D97FDFA95B1
:104540006283089508959C012A5F3F4FFC014281D8
:10455000461301C01282019682179307B9F7089596
:10456000262F2695269526952E3168F4FC01E20F1C
:10457000F11D677021E030E001C0220F6A95EAF773
:104580008281282B22830895262F2695269526950D
:104590002E3170F4FC01E20FF11D677021E030E074
:1045A00001C0220F6A95EAF7209582812823228391
:1045B000089520913401222329F02091470427FDFA
:1045C0000C94B0220C94892220913401222329F0EA
:1045D0002091470427FD0C94C4220C94A32220911F
:1045E0003401FC013296222331F08091470487FF89
:1045F00002C08EE101C086E0DF011D928A95E9F7D5
:10460000089508950C94012383E08093A5020C94EF
:104610000223811102C081E001C082E08093A502E3
:104620000C9402230C94092381E08093A5020C943E
:1046300002230C94142308950C941B230C941B2325
:10464000CF930E941E230E940A1F0E941C23C0E0D9
:104650008C2F0E94381E892B29F4CF5FC430C1F7FC
:1046600080E001C081E0CF910895089580916104B8
:10467000843011F00C94F10F08950E941A140C94D8
:10468000F30F82E084BD93E095BD9AEF97BD8093D0
:104690006E0008952FB7F8948091590490915A04B0
:1046A000A0915B04B0915C042FBF08952FB7F894DC
:1046B0006091590470915A0480915B0490915C045C
:1046C0002FBF08959C014FB7F894809159049091A1
:1046D0005A04A0915B04B0915C044FBF821B930B02
:1046E000089578941F920F920FB60F9211248F9312
:1046F0009F93AF93BF938091590490915A04A091D6
:104700005B04B0915C040196A11DB11D8093590416
:1047100090935A04A0935B04B0935C04BF91AF9153
:104720009F918F910F900FBE0F901F90189581E071
:104730008093E00080E28093D8001092C9008FE15E
:104740009EE40197F1F700C0000087E090EBDC01E8
:1047500080936A0490936B04A0936C04B0936D04EF
:104760009CE088E10FB6F894A895809360000FBE96
:1047700090936000FFCF8091C90208950895CF9370
:10478000DF9320913401222339F02091470427FF41
:1047900003C060E222E002C068E021E02093E9006B
:1047A0002FEF3091E800215035FD06C035ED3A95E8
:1047B000F1F700002111F5CF2091E80025FF1DC081
:1047C000EC0180913401811105C040E050E068E0C7
:1047D00070E003C070E040E050E0CE010E94E025B0
:1047E0008091E8008E778093E80080E2FE01A9EADC
:1047F000B2E001900D928A95E1F7DF91CF91089593
:104800008093A6027093A8026093A702809161042E
:10481000843001F582E08093E9008FEF9091E80009
:10482000815095FD06C095ED9A95F1F70000811134
:10483000F5CF8091E80085FF0DC040E050E063E0D7
:1048400070E086EA92E00E94E0258091E8008E7791
:104850008093E8000895BC0184E00C940024BC011E
:1048600083E00C940024089580916004811109C0B4
:104870000E9471270E94CE278091E200846080937D
:10488000E20008951092600408950C941923609139
:104890005D0481E0611101C080E00C9404239091DB
:1048A000610481E0943009F080E060915D040C9433
:1048B000092342E061EC81E00E94EA2642E261ECD9
:1048C00082E00E94EA269091610481E0943009F030
:1048D00080E060915D040C94122380916304833026
:1048E00009F461C030F4813071F0823009F49AC06B
:1048F00008958A3009F486C08B3009F46CC0893081
:1049000009F0A8C020C080916204813A09F0A2C0D9
:104910008091E800877F8093E80080916604909101
:104920006704892B21F460E289EA92E003C060E029
:1049300080E090E070E00E942B268091E8008B7769
:104940008093E800089580916204813209F082C06A
:104950008091660490916704029708F07BC0809173
:10496000E800877F8093E8008091E80082FD05C021
:10497000809161048111F8CF6DC02091F300809186
:10498000F20090E0922B029731F48091F100813097
:1049900011F0863021F48091F1008093C90280915A
:1049A000E8008B7753C080916204813A09F052C0CD
:1049B0008091660490916704892B09F04BC0809127
:1049C000E800877F8093E8008091E80080FFFCCFBB
:1049D0008091340136C0809162048132D9F5809192
:1049E000660490916704892BA9F58091E800877F80
:1049F0008093E8000E941F27809164048093340113
:104A00000C941A1480916204813221F58091E8009F
:104A1000877F8093E8000E941F2780916504809320
:104A2000CA02089580916204813AA1F48091E8005D
:104A3000877F8093E8008091E80080FFFCCF809121
:104A4000CA028093F1008091E8008E778093E8009D
:104A50000C941F27089584B7877F84BF0FB6F894FE
:104A6000A89580916000886180936000109260003A
:104A70000FBE90E080E80FB6F894809361009093A9
:104A800061000FBE0C9414230E9471270E94CE2750
:104A9000E2EEF0E080818460808378940C94632A55
:104AA00088E291E00C94EC21809161048530A9F4B6
:104AB00080916104853079F40E94362380915F04EF
:104AC0008823B1F30E942023882391F30E94CA25F2
:104AD0000E941A14EDCF0C943D23089508950C9470
:104AE0007125292F332723303105C9F060F4213097
:104AF000310581F02230310509F044C08BE390E0AC
:104B00002EE536E043C021323105E1F02232310595
:104B100049F138C082E190E029E936E037C09927B1
:104B20008130910549F028F0029761F5EEE1F6E059
:104B300005C0EAE5F6E002C0E2E4F6E0849190E028
:104B40009F0124C06115710541F061307105D1F4F8
:104B500089E090E029E836E019C089E090E020E79C
:104B600036E014C06115710541F06130710551F4F2
:104B70008DE690E02BEA36E009C080E490E028E181
:104B800037E004C080E090E020E030E0FA013183BB
:104B90002083089580E189BD82E189BD09B400FECA
:104BA000FDCF8091D8008F7D8093D8008091E00068
:104BB00082608093E0008091E00081FDFCCF089549
:104BC000CF92DF92EF92FF920F931F93CF93DF93D9
:104BD000EC018B017A010E943E27811133C0E11460
:104BE000F10439F0F70180819181081B190BC80F7E
:104BF000D91FC12CD12C0115110519F18091E800A4
:104C000085FD16C08091E8008E778093E800E1145E
:104C1000F10449F0F70180819181C80ED91ED1823B
:104C2000C08285E00FC00E943E27882321F30AC07E
:104C300089918093F10001501109FFEFCF1ADF0A2B
:104C4000DACF80E0DF91CF911F910F91FF90EF902D
:104C5000DF90CF9008952091680430916904261761
:104C6000370748F06115710539F42091E8002E7777
:104C70002093E80001C0B901FC0120E06115710535
:104C800079F1809161048823F1F18530F1F180910F
:104C9000E80083FD3CC08091E80082FD2EC0809139
:104CA000E80080FFEBCF2091F3008091F20090E0CC
:104CB000922B6115710551F08830910538F42191DE
:104CC0002093F100615071090196F3CF21E008971C
:104CD00009F020E08091E8008E778093E800CECF45
:104CE0002111CFCF0AC080916104882361F0853003
:104CF00061F08091E80083FD0AC08091E80082FFA6
:104D0000F2CF80E0089582E0089583E0089581E085
:104D1000089520916804309169042617370748F0F8
:104D20006115710539F42091E8002E772093E80091
:104D300001C0B901FC0120E06115710591F180917C
:104D40006104882309F440C0853009F43FC0809194
:104D5000E80083FD3DC08091E80082FD2FC0809176
:104D6000E80080FFE9CF2091F3008091F20090E00D
:104D7000922B6115710559F08830910540F424910A
:104D80002093F1003196615071090196F2CF21E034
:104D9000089709F020E08091E8008E778093E80082
:104DA000CBCF2111CCCF0AC080916104882361F060
:104DB000853061F08091E80083FD0AC08091E800B1
:104DC00082FFF2CF80E0089582E0089583E00895A5
:104DD00081E00895982F973068F59093E90098172F
:104DE00039F07091EC002091ED005091F00003C07B
:104DF000242F762F50E021FD02C09F5FECCF309131
:104E0000EB003E7F3093EB003091ED003D7F30931F
:104E1000ED003091EB0031603093EB007093EC00CB
:104E20002093ED005093F0002091EE0027FDE5CF98
:104E300080E008958F708093E90081E0089580916B
:104E4000620487FF11C08091E80082FD05C0809157
:104E500061048111F8CF11C08091E8008B770BC0FD
:104E600080916104882349F08091E80080FFF8CFA9
:104E70008091E8008E778093E80008952091E40007
:104E80003091E50095E64091EC00842F817040FF61
:104E900023C08091E80080FD1DC0809161048823BB
:104EA00099F0853099F08091EB0085FD11C040911B
:104EB000E4005091E5002417350729F3915011F0D3
:104EC0009A01E1CF84E0089582E0089583E0089597
:104ED00081E0089580E008954091E80042FFDDCF31
:104EE00008950E94DF270E94E727E0EEF0E080812E
:104EF00081608083E8EDF0E080818F77808319BC4A
:104F0000A7EDB0E08C918E7F8C9380818F7E808323
:104F10001092600408950F931F93CF93DF930E9424
:104F2000DF270E94E727C8EDD0E088818F7788834C
:104F300088818068888388818F7D888319BC1092DE
:104F4000610410925D0410925F0410925E0400EE02
:104F500010E0F80180818B7F808388818160888365
:104F600042E060E080E00E94EA26E1EEF0E080812D
:104F70008E7F8083E2EEF0E080818160808380819B
:104F800088608083F80180818E7F80838881806142
:104F90008883DF91CF911F910F910895E8EDF0E0A4
:104FA00080818F7E8083E7EDF0E080818160808367
:104FB00084E082BF81E0809360040C948B27E8ED4D
:104FC000F0E080818E7F80831092E200089510923D
:104FD000DA001092E10008951F920F920FB60F921F
:104FE00011242F933F934F935F936F937F938F93EE
:104FF0009F93AF93BF93EF93FF938091E10082FF64
:105000000BC08091E20082FF07C08091E1008B7F9E
:105010008093E1000E94622A8091DA0080FF1FC025
:105020008091D80080FF1BC08091DA008E7F809332
:10503000DA008091D90080FF0DC080E189BD82E156
:1050400089BD09B400FEFDCF81E0809361040E9418
:10505000342405C019BC109261040E94422480913E
:10506000E10080FF19C08091E20080FF15C08091AF
:10507000E2008E7F8093E2008091E2008061809365
:10508000E2008091D80080628093D80019BC85E04E
:10509000809361040E9447248091E10084FF30C026
:1050A0008091E20084FF2CC080E189BD82E189BD4E
:1050B00009B400FEFDCF8091D8008F7D8093D80089
:1050C0008091E1008F7E8093E1008091E2008F7EED
:1050D0008093E2008091E20081608093E200809101
:1050E0005D04882311F084E007C08091E30087FD10
:1050F00002C081E001C083E0809361040E944F24DC
:105100008091E10083FF29C08091E20083FF25C0E8
:105110008091E100877F8093E10082E080936104C9
:1051200010925D048091E1008E7F8093E100809178
:10513000E2008E7F8093E2008091E20080618093A4
:10514000E20042E060E080E00E94EA268091F00008
:1051500088608093F0000E944524FF91EF91BF91F9
:10516000AF919F918F917F916F915F914F913F91FF
:105170002F910F900FBE0F901F9018951F920F92B6
:105180000FB60F9211242F933F934F935F936F931A
:105190007F938F939F93AF93BF93CF93DF93EF93BF
:1051A000FF93C091E900CF708091EC00D82FD170AF
:1051B00080FDD0E81092E9008091F000877F809315
:1051C000F00078940E9402291092E9008091F0008A
:1051D00088608093F000CD2BCF70C093E900FF91E1
:1051E000EF91DF91CF91BF91AF919F918F917F917F
:1051F0006F915F914F913F912F910F900FBE0F9044
:105200001F9018951F93CF93DF93CDB7DEB7AA9762
:105210000FB6F894DEBF0FBECDBFE2E6F4E080919A
:10522000F100819324E0EA36F207C9F70E946D2469
:105230008091E80083FF2EC1809162049091630405
:10524000492F50E04A30510508F024C1FA01E558D1
:10525000FF4F0C94C82A803821F0823809F01AC117
:1052600008C080915E0490915F04992389F0826068
:105270000FC0809166048F70873008F00BC1809357
:10528000E9008091EB0085FB882780F91092E90006
:105290009091E800977F9093E8008093F10010923E
:1052A000F100D1C0282F2D7F09F0F4C0882319F018
:1052B000823061F0EFC080916404813009F0EAC06F
:1052C000933009F080E080935F042EC080916404E5
:1052D00081112AC0809166048F702FEF280F26302D
:1052E00008F0D8C08093E9002091EB0020FF1CC09B
:1052F000933021F48091EB00806214C09091EB0018
:1053000090619093EB0021E030E0A90102C0440FCE
:10531000551F8A95E2F74093EA001092EA008091C7
:10532000EB0088608093EB001092E9008091E80028
:10533000877F8093E8000E941F27ACC08111AAC01C
:10534000109164041F778091E3008078812B809313
:10535000E3008091E800877F8093E8000E941F2788
:105360008091E80080FFFCCF8091E300806880930B
:10537000E300111102C082E001C083E08093610468
:1053800089C08058823008F085C080916404909173
:1053900065048C3D53E0950779F583E08A838AE2C2
:1053A00089834FB7F894DE01139620E03EE051E286
:1053B000E32FF0E050935700E49120FF03C0E29503
:1053C000EF703F5FEF708E2F90E0EA3010F0C796DD
:1053D00001C0C0968D939D932F5F243149F74FBF35
:1053E0008091E800877F8093E8006AE270E0CE0158
:1053F00001960E942B2616C0609166047091670486
:10540000AE014F5F5F4F0E946F25BC01892B09F4ED
:1054100041C09091E800977F9093E80089819A813C
:105420000E9489268091E8008B778093E80032C043
:10543000803881F58091E800877F8093E800809133
:105440005D048093F1008091E8008E7772CF811126
:1054500021C0809164049091650499270297D4F447
:105460008091E800877F8093E800809164048093B6
:105470005D040E941F2780915D04811106C0809108
:10548000E30087FD02C081E001C084E080936104F5
:105490000E9459248091E80083FF0AC08091E800AF
:1054A000877F8093E8008091EB0080628093EB001F
:1054B000AA960FB6F894DEBF0FBECDBFDF91CF9195
:1054C0001F9108950895CF93809161048823A1F0DE
:1054D000C091E900CF709091EC00892F817090FD10
:1054E00080E8C82B1092E9008091E80083FD0E94BB
:1054F0000229CF70C093E900CF910895AA1BBB1B6E
:1055000051E107C0AA1FBB1FA617B70710F0A61BC3
:10551000B70B881F991F5A95A9F780959095BC01E4
:10552000CD01089597FB072E16F4009407D077FD60
:1055300009D00E947E2A07FC05D03EF49095819503
:105540009F4F0895709561957F4F0895A1E21A2E9F
:10555000AA1BBB1BFD010DC0AA1FBB1FEE1FFF1F17
:10556000A217B307E407F50720F0A21BB30BE40B67
:10557000F50B661F771F881F991F1A9469F76095AE
:105580007095809590959B01AC01BD01CF01089568
:10559000EE0FFF1F0590F491E02D09948F929F92DA
:1055A000AF92BF92CF92DF92EF92FF92CF93DF93B1
:1055B000EC01688179818A819B8161157105810582
:1055C000910521F464E279ED8BE597E02DE133EF6D
:1055D00041E050E00E94922B49015A019B01AC012D
:1055E000A7EAB1E40E94B12B6B017C01ACEEB4EFF1
:1055F000A50194010E94BF2BDC01CB018C0D9D1DE8
:10560000AE1DBF1DB7FF03C00197A109B048888335
:105610009983AA83BB839F77DF91CF91FF90EF900F
:10562000DF90CF90BF90AF909F908F9008950E9491
:10563000CE2A089580E091E00E94CE2A0895A0E04D
:10564000B0E08093000190930101A0930201B09318
:1056500003010895FB01DC0102C005900D92415049
:105660005040D8F70895FB01DC0104C08D910190F2
:10567000801921F441505040C8F7881B990B0895B8
:10568000DC01CB01FC01F999FECF06C0F2BDE1BD02
:10569000F89A319600B40D9241505040B8F70895F1
:1056A000F999FECF92BD81BDF89A992780B50895EA
:1056B000A8E1B0E042E050E00C94422BDC01A40FE2
:1056C000B51F4150504048F0CB01840F951F2E91DB
:1056D0000E946F2B41505040D0F70895262FF99922
:1056E000FECF92BD81BDF89A019700B4021639F041
:1056F0001FBA20BD0FB6F894FA9AF99A0FBE089512
:105700000396272F0E946F2B0E946E2B252F0E943D
:105710006F2B242F0C946F2B0196272F0E946F2B39
:105720000C946E2B052E97FB1EF400940E94A92B5F
:1057300057FD07D00E94A62A07FC03D04EF40C9414
:10574000A92B50954095309521953F4F4F4F5F4F76
:10575000089590958095709561957F4F8F4F9F4FDD
:1057600008950E94C42BA59F900DB49F900DA49FF7
:10577000800D911D11240895B7FF0C94B12B0E9448
:10578000B12B821B930B0895A29FB001B39FC00160
:10579000A39F700D811D1124911DB29F700D811D5D
:0A57A0001124911D0895F894FFCF25
:1057AA0001000000FF0000FFFF0000FF7FFF000074
:1057BA00FF0000FF0000FF0000FF031003100310AA
:1057CA00FF1F0000C8006502BB23BF2333242F2418
:1057DA002B24BE2301E200E900EA00B500B600B7B7
:1057EA0000CD008301CC008A019201940121022399
:1057FA000224022502260227022A02B300B4006FFD
:10580A00007000818283E200E900EA00B500B60078
:10581A00B700CD008301CC008A01920194012102D4
:10582A00230224022502260227022A02B300B40018
:10583A006F007000818283F4356766363233313403
:08584A0097969493F0F1F5F636
:00000001FF
